:100000000C9467030C94AB030C94AB030C94AB03FC
:100010000C94AB030C94AB030C94AB030C94AB03A8
:100020000C94AB030C94AB030C946A150C943C1623
:100030000C949E230C94AB030C94AB030C94AB0375
:100040000C94AB030C940D040C94AB030C94AB0315
:100050000C94AB030C9406240C94AB030C94AB03EC
:100060000C94AB030C94AB030C94AB030C94AB0358
:100070000C94AB030C94AB030C94AB030C94AB0348
:100080000C94DF0B0C94AB030C94AB030C94AB03FC
:100090000C94AB030C94AB030C94AB030C94AB0328
:1000A0000C94AB030C94AB030C94AB03A916CB16C6
:1000B000B917CB16B91710173317B91788179B172D
:1000C000851A851AB41AB41AF31A131B691C691C11
:1000D0001E1B691CCE1BCE1B351C3E1C691C631CE1
:1000E000DB1BDB1BDB1BDB1BDB1BDB1BDB1BDB1B60
:1000F000DB1BDB1BDB1BDB1BDB1BDB1BDB1BDB1B50
:10010000EB1BF91B001C071C111C07634236B79B35
:10011000D8A71A39685618AEBAAB558C1D3CB7CC67
:100120005763BD6DEDFD753EF6177231BF000000DF
:10013000803F08000000BE922449123EABAAAA2AC2
:10014000BECDCCCC4C3E00000080BEABAAAAAA3EDD
:1001500000000000BF000000803F00000000000819
:100160004178D3BB4387D1133D190E3CC3BD4282B6
:10017000AD2B3E68EC8276BED98FE1A93E4C80EF74
:10018000FFBE01C4FF7F3F00000000000000000030
:1001900000000000000000010204060A0F17202CD6
:1001A0003A4A5D71879DB3C7DAE9F5FCFFFCF5E9D2
:1001B000DAC7B39D87715D4A3A2C20170F0A0604EF
:1001C00002010000000000000000000001E1013316
:1001D000023301260226012C022C012C022C0127BD
:1001E00002270133023302E1015002500150025054
:1001F000015002500001E1012602260133023301C1
:100200002C022C012C022C0133023301270227027D
:10021000E10150025001500250015002500001E132
:10022000013302330126022602E10001E10133021B
:10023000330127022702E1000000F1A4F1A529A65D
:1002400000000000018C028C048C088C000000006F
:100250000000000000002B22032014001A000900F7
:1002600013000A000D000F0018001C0033002D00C1
:100270002A00040015001600170007000B001100EB
:1002800008000C00120028000F201D001B000600B3
:10029000190005000E00100036003700520034002F
:1002A000E000E300E200E10001202C002C0002202D
:1002B0003800500051004F00032014001A000800BD
:1002C000150017001C0018000C00120013002D0070
:1002D0002A0004001600070009000A000B000D00A8
:1002E0000E000F00330028000F201D001B00060029
:1002F00019000500110010003600370052003400CC
:10030000E000E300E200E10001202C002C000220CC
:100310003800500051004F00032000005200000040
:10032000000000002602270254005F006000610008
:100330002A00500051004F00000000002202670018
:1003400055005C005D005E000F2000000000000012
:100350000000000000008500560059005A005B00B4
:10036000E000E300E200E1000120010001000220C2
:100370005700620063005800032014001A000900AF
:10038000130023000D000F0018001C0033002D0087
:100390002A00210015002200240007000B00110094
:1003A00020001E00270028000F201D001B00060053
:1003B000190005000E00100036003700520034000E
:1003C000E000E300E200E10001202C002C0002200C
:1003D0003800500051004F003500000000000000C0
:1003E0000000000000000000033002300130003047
:1003F0002A001E001F0020002100220023002400EC
:100400002500260027000100310000000000000048
:1004100000000000000000002F0030004B002E0004
:100420000100010001000100012001000100022083
:1004300000004A004E004D003A003B003C003D00E9
:100440003E003F00400041004200430044004500A0
:100450004C00F400F000F500F600F900F700500041
:10046000510052004F0000000100F200F100F300C3
:10047000FB00FA00FC00000000004B0152054E0199
:100480000100010001000100012000000000022025
:100490000000500551054F050100A800AA00A90061
:1004A000000000000000000000000000000000004C
:1004B0000000AE00AC00AB00000000000000000037
:1004C00000000000000000500000000000000000DC
:1004D000000000000000000000000000000000001C
:1004E0000620072008200920012001000100022029
:1004F0006600A700A6000F052803540068006500E9
:10050000200050006C0061006E0063006B00200052
:100510004B006500790062006F00610072006400AA
:1005200000002C034F007200740068006F006C0024
:1005300069006E0065006100720020004B006500DC
:10054000790062006F0061007200640073000000B7
:100550000403090409026D00040100A0FA09040063
:10056000000103010100092111010001223F0007E0
:1005700005810308000A09040100010301020009C2
:100580002111010001224D000705820308000A091C
:1005900004020001030000000921110100012236BC
:1005A000000705830308000A090403000103000093
:1005B0000009211101000122390007058403100000
:1005C000011201100100000008EDFE606001000151
:1005D00002000105010906A101050719E029E71537
:1005E0000025019508750181020508190129059565
:1005F00005750191029501750391010507190029FF
:100600007715002501957875018102C005010980E3
:10061000A101850216010026B7001A01002AB700C1
:10062000751095018100C0050C0901A10185031613
:100630000100269C021A01002A9C02751095018176
:1006400000C005010902A1010901A1000509190164
:100650002905150025019505750181029501750390
:1006600081010501093009311581257F9502750841
:10067000810609381581257F950175088106050CCD
:100680000A38021581257F950175088106C0C005CD
:10069000010906A101050719E029E71500250195C3
:1006A0000875018102950175088101050819012964
:1006B00005950575019102950175039101050719CD
:1006C0000029FF150025FF950675088100C011243B
:1006D0001FBECFEFDAE0DEBFCDBF04B603FE24C0FD
:1006E00080911E0390911F03A0912003B0912103DC
:1006F0008730904BA740B04BB9F410921E03109274
:100700001F03109220031092210314BE84B7877F29
:1007100084BF88E10FB6F894809360001092600067
:100720000FBEE0E0F8E3099511E0A0E0B1E0E6E9F2
:10073000FBE502C005900D92A03CB107D9F713E08C
:10074000A0ECB1E001C01D92AE31B107E1F70E940B
:10075000B0120C94C92D0C9400000895089581E006
:10076000089508950C94AE030C94AF030C94B10358
:100770000E94932923E030E0281B3109220F2093A7
:10078000C4010895282F2F9880918000211108C05E
:10079000877F8093800010928D0010928C001BC088
:1007A000886080938000233019F48FEF9FEF0FC093
:1007B00083E090E0821B9109880F991F2FEF3FEF94
:1007C000A90102C0569547958A95E2F7CA01909310
:1007D0008D0080938C000C94B8030E94B80384E0D1
:1007E0008093C3011092C0010895279A2F988FEF2C
:1007F0009FEF90938700809386008AE0809380002B
:1008000089E1809381000E94FC280C94ED030E94F2
:10081000F5036E9A769A0C94AD031F920F920FB661
:100820000F9211242F933F938F939F93EF93FF93F6
:10083000E091C101F091C201CF0101969093C201F4
:100840008093C1010090C30102C0F695E7950A9418
:10085000E2F7EF738091C001823019F4E03251F475
:1008600004C0813039F4EF3329F480916F008D7F1B
:1008700080936F00F0E0E457FE4FE49121E031E017
:10088000E29FC001E39F900D11240090C40102C0BB
:10089000969587950A94E2F790938D0080938C004B
:1008A000FF91EF919F918F913F912F910F900FBEEC
:1008B0000F901F901895FC01613061F028F06230B4
:1008C00079F0633099F018C082818823A9F08BE217
:1008D00092E008958281882379F08EE192E0089574
:1008E0008281882349F085EF91E0089582818823F1
:1008F00019F08CEC91E0089580E090E0089581E09B
:1009000008950C947F0408950C94070480911502B7
:10091000882309F448C08091D1019091D2010097B9
:1009200079F40E94D0239093D2018093D1018091D9
:10093000D30190E0009771F48091D40190E00AC057
:100940000E94DC2320910001309101012817390712
:1009500040F329C00197880F991F880F991FFC0148
:10096000EB52FE4F60817181828193810E94450B21
:10097000E091D30184E0E89FF0011124EB52FE4F97
:1009800060817181828193814FE050E00E94FD0E71
:100990008091D30190E001966091D40170E00E94B3
:1009A000792D8093D3010C94B203109217020C940A
:1009B000120B0895089581E0809317020C94DA04D5
:1009C000089508958F929F92AF92BF92EF92FF92F7
:1009D0000F931F93CF93DF93CDB7DEB7A3970FB6D7
:1009E000F894DEBF0FBECDBF7C01FC0100811181F8
:1009F000C8010E94CD21B8010E94E4068C01B70114
:100A00000E948104882309F4CCC10032F0E51F075D
:100A100041F4F7018281882309F458C00E94610FD4
:100A2000C0C10132F0E51F0741F4F701828188233C
:100A300009F44CC00E946A0FB4C10232F0E51F07EE
:100A400051F4F7018281882309F440C00E945D0FB0
:100A50008111F0CFE3CF0332F0E51F0739F4F7013E
:100A60008281882399F10E94DB049BC10432F0E566
:100A70001F0739F4F7018281882341F10E94D504D0
:100A800090C10532F0E51F0749F4F7018281882300
:100A9000E9F0809117028111F1CFE5CF0632F0E540
:100AA0001F0739F4F7018281882381F00E94710FBA
:100AB0000AC00732F0E51F0749F4F7018281882355
:100AC00029F00E947C0F0E94E1046BC18091170203
:100AD000811105C0F70182818111CFC018C1003E8C
:100AE000110579F4F7018281882309F44DC00E9431
:100AF000120B81E080931602109215021092D4011D
:100B000050C1023E110559F4F70182818823E1F1B9
:100B10000E94120B109216021092150242C1033E5F
:100B2000110591F4F7018281882371F10E94120B63
:100B30001092160281E0809315021092D301109258
:100B4000D2011092D1012DC10235110559F4F701DE
:100B50008281882309F425C18091000190910101CF
:100B60000A970DC00135110579F4F70182818823B8
:100B700009F417C180910001909101010A969093A8
:100B80000101809300010DC14091040183E2EFE176
:100B9000F1E0DE01119601900D928A95E1F7F701DF
:100BA000808121E030E02C0F3D1F280F311DC9014D
:100BB0002091020130910301FC01E20FF31F6081DB
:100BC000772767FD7095640F711D882777FD8095E5
:100BD000982F0E949B2A20E030E040E451E40E94DC
:100BE000002A4B015C01F701218184E090E0821B27
:100BF0009109BC01882777FD8095982F0E949B2A38
:100C00009B01AC01C501B4010E9498299B01AC0174
:100C100060E070E080E090E40E940E2C20E030E084
:100C20004CED50E40E94AB2B4B015C01F70182813B
:100C30008823D1F04FE050E0C501B4010E94FD0EC1
:100C4000809116028823A1F08091D40124E0829F34
:100C5000F0011124EB52FE4F80829182A282B38276
:100C60008F5F8093D40104C0C501B4010E94450B7D
:100C70000F3F110508F02ECF94C08091D001811153
:100C80001FC0043130E5130709F051C00E948304EE
:100C900081E08093D0010E94D0239093CF01809374
:100CA000CE011092C7011092C9011092C801109292
:100CB000CB011092CA011092CD011092CC0171C0EB
:100CC0008091CE019091CF010E94DC23883C910558
:100CD00070F48091C701E82FF0E0EE0FFF1FE8539A
:100CE000FE4F118300838F5F8093C7015AC0043881
:100CF00080E5180721F00538104501F13AC0F701E9
:100D00008281882341F01092C50182E01EC0043820
:100D100030E5130759F58091C501811106C086E2BF
:100D20000E94291986E20E94F11982E01CC0043851
:100D3000F0E51F0741F305381045D9F4F70182812A
:100D4000882331F01092C60180E20E94401A29C027
:100D50008091C601811106C087E20E94291987E2AD
:100D60000E94F11980E20E94471A1BC00538104505
:100D700029F381E08093C5018093C601C701A39642
:100D80000FB6F894DEBF0FBECDBFDF91CF911F919C
:100D90000F91FF90EF90BF90AF909F908F900C9429
:100DA000B40380E0A3960FB6F894DEBF0FBECDBFAC
:100DB000DF91CF911F910F91FF90EF90BF90AF9077
:100DC0009F908F90089508959CE0799FF0011124E1
:100DD00090E3899FE00DF11D1124E60FF11DEE0F48
:100DE000FF1FE85AFD4F859194910895880F991F30
:100DF000FC01E854FF4F859194910895880F991F45
:100E0000FC01E85CFD4F8591949108950F931F9329
:100E1000CF93DF93EC01811521E39207A0F5C11573
:100E200080E3D80708F0D7C0C83ED105D8F4C03E4B
:100E3000D10508F007C2C83AD10578F4C53AD10502
:100E400008F06AC0C130D10509F463C008F4F7C1E5
:100E5000C430D10508F0F6C1F2C1CB3BD10508F48E
:100E600066C0EDC1C11590E2D90708F0AFC0C11549
:100E700021E0D20708F0E6C1C03FD10508F4DFC188
:100E80008E0110651FC2C03880E5D80700F5C03755
:100E900090E5D90708F0A3C0C11520E5D20709F4F1
:100EA000ACC050F4CE01905480319F4008F0C7C1CF
:100EB000DF708E01106A06C2C13080E5D80709F4E0
:100EC000AEC0C43190E5D90708F4AFC0B8C1C3388B
:100ED00020E5D20709F48EC050F4C13890E5D90757
:100EE00009F482C008F083C000E011EDEBC1C0310D
:100EF00081E5D80708F4A3C1C11597E5D90708F41F
:100F000036C1CE0190578115904108F098C1DF702D
:100F100093C101E010E0D6C1C53AD10509F494C1EE
:100F2000C63AD10509F093C102E810E4CBC1C83A32
:100F3000D10509F48FC1C93AD10509F48EC1CA3A65
:100F4000D10509F48DC1CB3AD10509F48CC1CC3A55
:100F5000D10509F48BC1CD3AD10509F48AC1C03B52
:100F6000D10509F489C1CE3AD10509F488C1CF3A37
:100F7000D10509F487C1C13BD10509F486C1C23B43
:100F8000D10509F485C1C33BD10509F484C1C43B33
:100F9000D10509F483C1C53BD10509F482C1C63B23
:100FA000D10509F481C1C73BD10509F480C1C83B13
:100FB000D10509F47FC1C93BD10509F47EC1CA3B03
:100FC000D10509F47DC100E014E47CC1CE019F701D
:100FD0000E94FE0678C1DD278E01106C73C1CF70B0
:100FE000DD278E01146D6EC100E010ED6BC100E0D5
:100FF00012ED68C100E013ED65C10E94D41C0E948F
:10100000120B0E94D9048FEF94E32CE081509040A2
:101010002040E1F700C000000E942B2453C18091C2
:10102000F20281608093F2024DC10E948C248111F2
:1010300002C00E9468240E949F2490E090931D03A8
:1010400080931C03C23080E5D80721F480911C03F3
:10105000816086C0C43090E5D90721F480911C03DB
:1010600082607EC0C63020E5D20721F480911C0347
:10107000846076C0C83080E5D80719F480911C03DD
:1010800027C0CA3090E5D90721F480911C03806104
:1010900067C0CC3020E5D20721F480911C03806228
:1010A0005FC0CE3080E5D80721F480911C038064B6
:1010B00057C0C03190E5D90721F480911C038068A6
:1010C0004FC0C23120E5D20729F480911C0384600F
:1010D000886046C0C33080E5D80721F480911C03A6
:1010E0008E7F3EC0C53090E5D90721F480911C0366
:1010F0008D7F36C0C73020E5D20721F480911C03D4
:101100008B7F2EC0C93080E5D80719F480911C036D
:1011100026C0CB3090E5D90721F480911C038F7E47
:101120001FC0CD3020E5D20721F480911C038F7DB4
:1011300017C0CF3080E5D80721F480911C038F7B46
:101140000FC0C13190E5D90721F480911C038F773E
:1011500007C0C331D04531F480911C038B7F877F5A
:1011600080931C0380911C030E94A324ABC08D2F8D
:1011700099278F70992781309105D9F49E012370AA
:10118000332702C0880F991F2A95E2F79C688E01C9
:1011900044E0000F111F4A95E1F700271370802BE0
:1011A000912B53E0CC0FDD1F5A95E1F7C076DD2778
:1011B0002FC08230910531F4DC2FCC278E01016FD6
:1011C000106A80C08330910569F4CE01837099273D
:1011D00001E010E002C0000F111F8A95E2F7C8017C
:1011E0009C680FC084309105B9F4CE0183709927B3
:1011F00001E010E002C0000F111F8A95E2F7C8015C
:101200009A6823E0CC0FDD1F2A95E1F7C07ED770E6
:101210008C010C2B1D2B56C08530910531F4DC2F31
:10122000CC278E01046F106A4DC0069709F04AC0A2
:10123000CF71DD27DC2FCC278E01106243C000E088
:1012400010E040C08E013EC001E810E43BC003E85E
:1012500010E438C002EE14E435C009EE14E432C0E4
:101260000AEE14E42FC005EB14E42CC006EB14E4E2
:1012700029C007EB14E426C00CEC14E423C00DECE9
:1012800014E420C003E815E41DC00AE815E41AC000
:1012900002E915E417C004E915E414C001E216E4FC
:1012A00011C003E216E40EC004E216E40BC005E22E
:1012B00016E408C006E216E405C007E216E402C020
:1012C0000AE216E4C801DF91CF911F910F910895B2
:1012D0009CE0799FF001112490E3899FE00DF11DBE
:1012E0001124E60FF11DEE0FFF1FE85AFD4F859107
:1012F0009491803E9105E0F4803C910558F581334E
:10130000910509F46FC048F48932910509F463C06E
:101310008A32910509F46DC072C089339105E9F0F4
:1013200082389105D1F08533910509F44DC067C02D
:10133000833E910581F138F4803E9105B9F0823EFB
:101340009105D9F05CC0863E910561F1873E91051B
:10135000A1F155C00E94F606089520911C0320FDBE
:1013600002C021FF4CC080EE90E049C080911C0378
:1013700080FFF9CF89E390E042C080911C0382FF97
:101380000EC080911C0384FF03C080E090E037C052
:1013900083EE90E034C080911C0382FFF2CF82EE96
:1013A00090E02DC080911C0383FF0BC080911C0333
:1013B00084FDEBCF87EE90E022C080911C0383FF79
:1013C000F5CF86EE90E01BC080911C0385FF07C01F
:1013D00089E290E014C080911C0385FFF9CF85E37A
:1013E00090E00DC080911C0386FF07C08AE290E068
:1013F00006C080911C0386FFF9CF81E390E00E9434
:10140000060708950C94B603E82FF0E0E25BFE4F68
:101410008081E82FEF70F0E082958F7021E030E05E
:10142000A90102C0440F551F8A95E2F740A3089511
:101430000F931F93CF93DF9385B7806885BF85B7E0
:10144000806885BFC3E0D0E001E010E0FE01E25B10
:10145000FE4F8081E82FEF70F0E021A182958F7020
:10146000A80102C0440F551F8A95E2F7CA01822BDA
:1014700081A38C2F0E94040A219740F78BE090E013
:1014800061E070E0FC01EE5BFE4F2081E22FEF7027
:10149000F0E042A122952F70DB0102C0AA0FBB1F12
:1014A0002A95E2F79D01242B22A3019758F7DF919B
:1014B000CF911F910F910C948404EF92FF920F93A0
:1014C0001F93CF93DF9300E212E0C3E0EE24E39496
:1014D000F12CD5E08C2F0E94040A8BE090E040E0D4
:1014E00050E0FC01EE5BFE4F6081E62FEF70F0E014
:1014F00020A130E062956F7002C0359527956A95FE
:10150000E2F720FD09C09701082E02C0220F331F09
:101510000A94E2F7422B532B019718F7F8019291A6
:1015200082918F018417950721F051834083D093D6
:1015300005018C2F0E94040AC15060F680910501BC
:1015400087FD2CC08150809305018F3F39F08FE9D2
:101550009FE00197F1F700C0000020C080911E02BB
:1015600090911F02909327028093260280911C0283
:1015700090911D02909325028093240280911A027B
:1015800090911B0290932302809322028091180273
:101590009091190290932102809320020E94860468
:1015A00081E0DF91CF911F910F91FF90EF9008950F
:1015B000E82FF0E0EE0FFF1FE05EFD4F808191818C
:1015C000089508950F931F93CF9308E212E0C0E0AF
:1015D000F801929182918F010E944823C80FF2E096
:1015E00000321F07A9F78C2FCF911F910F910895FB
:1015F0000E948C24811102C00E9468240E94B124A0
:10160000809307033E9A809171008D7F80937100D3
:1016100082E0809390008AE18093910081E0809342
:101620002A02089580912A02811102C00E94F80ABC
:1016300010927A0210927902809171008D7F8093CE
:101640007100809190008F738093900010923C0203
:1016500010923B0210927302109274021092750263
:10166000109276021092720210927102E1E5F2E09D
:10167000A1E4B2E011921192119211921D921D9269
:1016800082E0E137F807B1F70895CF92DF92EF9249
:10169000FF920F931F93CF93DF9320913B0222235E
:1016A00009F484C06B017C0180912A02811102C07F
:1016B0000E94F80A01E712E0C7E0D0E0A701960116
:1016C000F80192918291729162918F010E94FC299E
:1016D000811131C0FE01EE0FFF1FEE0FFF1FEF5A09
:1016E000FD4F1082118212821382DE01AA0FBB1FEE
:1016F000AF5BBD4F11961C921E92C730D105E9F029
:10170000219644815581668177814083518362832C
:101710007383148215821682178212968D919C9182
:10172000139711969C938E9313961C921E92129768
:1017300034961296E2CF219708F680917902909123
:101740007A02019797FD05C090937A0280937902FF
:1017500004C010927A0210927902809179029091DD
:101760007A0220917702309178022817390724F005
:101770001092780210927702892BC1F48091710047
:101780008D7F80937100809190008F738093900083
:1017900010927302109274021092750210927602E7
:1017A000109272021092710210923B02DF91CF915F
:1017B0001F910F91FF90EF90DF90CF9008951F92AF
:1017C0000F920FB60F9211244F925F926F927F92F9
:1017D0008F929F92AF92BF92CF92DF92EF92FF9241
:1017E0002F933F934F935F936F937F938F939F9329
:1017F000AF93BF93CF93DF93EF93FF9380913B021F
:10180000882309F49BC1C0917902D0917A021C16F9
:101810001D060CF093C140902B0250902C0260905A
:101820002D0270902E0220E030E0A901C301B20128
:101830000E94A72B18160CF065C0C130D10509F421
:1018400052C08091770290917802BE010E94792D5A
:101850007C01909378028093770280903D02909073
:101860003E02A0903F02B090400220E030E040E80D
:101870005FE3C501B4010E94982960933D02709313
:101880003E0280933F0290934002F701EE0FFF1F4C
:10189000EE0FFF1FEF5AFD4FA3019201608171818E
:1018A000828193810E94002A20E030E040E05EE3E4
:1018B0000E94AB2B9B01AC01C501B4010E94A72B78
:1018C00018168CF4C7010196BE010E94792D9093E1
:1018D00078028093770210923D0210923E0210929D
:1018E0003F0210924002E0917702F0917802EE0FF1
:1018F000FF1FEE0FFF1FEF5AFD4F60817181828144
:101900009381D0C0C0907302D0907402E0907502B1
:10191000F090760220E030E0A901C701B6010E94F4
:10192000FC292197882309F4A2C0FE01EE0FFF1FB6
:10193000EE0FFF1FEF5AFD4F80809180A280B38091
:10194000A5019401C701B6010E94FC2987FF31C09F
:10195000A501940160E070E08CED93EC0E94002AF8
:1019600020E030E040E451E40E94002A20E030E032
:1019700040E05FE30E94AB2B9B01AC0160E070E0B4
:1019800080E090E40E940E2C9B01AC01C501B401E3
:101990000E94AB2B9B01AC01C701B6010E94FC2940
:1019A00087FF07C0A701960160E070E08CED93E42B
:1019B00039C0A5019401C701B6010E94A72B1816D2
:1019C0000CF055C0A501940160E070E08CED93E44B
:1019D0000E94002A20E030E040E451E40E94002A06
:1019E00020E030E040E05FE30E94AB2B9B01AC01C4
:1019F00060E070E080E090E40E940E2C9B01AC015E
:101A0000C501B4010E94AB2B9B01AC01C701B6011B
:101A10000E94A72B18165CF5A701960160E070E004
:101A20008CED93EC0E94002A20E030E040E451E489
:101A30000E94002A20E030E040E05FE30E94AB2BF0
:101A40009B01AC0160E070E080E090E40E940E2C0D
:101A50009B01AC01C701B6010E94AB2B60937302DE
:101A600070937402809375029093760213C0FE0106
:101A7000EE0FFF1FEE0FFF1FEF5AFD4F8081918188
:101A8000A281B3818093730290937402A093750234
:101A9000B093760260917302709174028091750226
:101AA0009091760220912802309129022F3F4FEF2A
:101AB000340731F02F5F3F4F3093290220932802E3
:101AC0000E94870F6B017C0120E034E244EF51E477
:101AD0000E94FC2987FF08C086EFC82E88E2D82E16
:101AE00084EFE82E81E4F82E20E030E040E051E47D
:101AF000C701B6010E94AB2B9B01AC0160E074E210
:101B000084E79BE40E94002A6B017C010E946D2AFD
:101B10007093970060939600209106013091070121
:101B20004091080150910901C701B6010E94AB2BF9
:101B30000E946D2A709399006093980080913C02F6
:101B4000882309F433C1C0903702D0903802E09066
:101B50003902F0903A0220E030E0A901C701B60155
:101B60000E94A72B1816D4F5809128029091290283
:101B70008F3F2FEF920729F00196909329028093CF
:101B80002802C701B6010E94870F20E030E040E044
:101B900051E40E94AB2B9B01AC0160E074E284E74E
:101BA0009BE40E94002A6B017C010E946D2A7093C5
:101BB00097006093960020910601309107014091B3
:101BC000080150910901C701B6010E94AB2B0E9488
:101BD0006D2A709399006093980008C01092970046
:101BE0001092960010929900109298006091310224
:101BF000709132026F5F7F4F7093320260933102B7
:101C0000209196003091970080E090E0232BF1F036
:101C1000C0919600D09197000E94992A6B017C0197
:101C2000BE0180E090E00E94992A9B01AC01609186
:101C300033027091340280913502909136020E94F5
:101C4000002A20E03FEF4FE757E410C00E94992A96
:101C50006B017C0120E030EE4FEF54E460913302E1
:101C60007091340280913502909136020E94AB2B24
:101C70009B01AC01C701B6010E94A72B87FD96C04E
:101C800080912F028F5F80932F0290E020910303B9
:101C90003091040382179307A0F080910E038823EC
:101CA00019F010922F020DC0809171008D7F8093EA
:101CB0007100809190008F738093900010923C028D
:101CC0007DC080913002C0912F02811128C0C09048
:101CD0000803D0900903E0900A03F0900B0320E082
:101CE00030E0A901C701B6010E94A72B1816BCF469
:101CF00081E08093300210923702109238021092E5
:101D0000390210923A02C0923302D0923402E09229
:101D10003502F0923602C150C0932F0243C0109298
:101D200030021092290210922802E0910503F091EE
:101D3000060348E0C49FE00DF11D112480819181CC
:101D4000A281B3818093370290933802A093390225
:101D5000B0933A0220E030E040E85EE364817581B0
:101D6000868197810E94AB2B6B017C0180910A01D7
:101D7000682F70E080E090E00E94992A20E030E037
:101D800048EC52E40E94002A9B01AC01C701B60155
:101D90000E94AB2B60933302709334028093350220
:101DA0009093360210923202109231028091070312
:101DB00080FD04C010923C0210923B02FF91EF9113
:101DC000DF91CF91BF91AF919F918F917F916F9153
:101DD0005F914F913F912F91FF90EF90DF90CF90C7
:101DE000BF90AF909F908F907F906F905F904F903B
:101DF0000F900FBE0F901F901895CF92DF92EF9229
:101E0000FF92CF93DF936B017C01EA0180912A025C
:101E1000811102C00E94F80A8091070380FF46C02A
:101E20008091790290917A0208970CF03FC08091DE
:101E300071008D7F8093710080913C0281110E941E
:101E4000120B81E080933B0210922902109228022B
:101E500020E030E0A901C701B6010E94A72B1816A7
:101E6000DCF48091790290917A02FC01EE0FFF1F61
:101E7000EE0FFF1FEF5AFD4FC082D182E282F38244
:101E8000FC01EE0FFF1FEF5BFD4FD183C083019676
:101E900090937A028093790280917100826080939E
:101EA000710080919000806880939000DF91CF91C5
:101EB000FF90EF90DF90CF9008958091070381709D
:101EC0000895809107038160809307030E94B524E1
:101ED0000C94E004809107038E7F809307030C9499
:101EE000B52480917B0290E0019666E070E00E944C
:101EF000792D80937B02089580917B0290E0019779
:101F000066E070E00E94792D80937B0208958F92A5
:101F10009F92AF92BF92CF92DF92EF92FF920F9378
:101F20001F93CF93DF936B017C01C0912802D09166
:101F30002902BE0180E090E00E94992A4B015C01D9
:101F4000A701960160E070E08CE594E40E94002A0D
:101F50009B01AC01C501B4010E94AB2B0E946D2A0C
:101F600020917B02233009F473C028F4222351F01E
:101F70002130E9F02CC1243009F4A0C0253009F447
:101F8000E0C025C180E090E0A0E0BFE380930601BF
:101F900090930701A0930801B093090110922B02BE
:101FA00010922C0210922D0210922E0210C110924B
:101FB0002B0210922C0210922D0210922E026431EC
:101FC000710540F46A30710560F520E030E040E8CA
:101FD0005EE32BC0693C710508F0AAC080E090E088
:101FE0000E94992A20E030E040EA51E40E949729BB
:101FF00020E030E044E353E40E94002A9B01AC015E
:102000000E94AB2B20E030E040E05EE30E94AB2B6F
:102010009B01AC0160E070E080E09EE30E949729A4
:1020200044C020E030E040E05FE3C701B6010E9419
:10203000AB2B6B017C0180E090E0A0E0BEE38093DD
:10204000060190930701A0930801B0930901BFC056
:1020500010922B0210922C0210922D0210922E023E
:102060004AE0469F9001479F300D1124C90168EB5B
:102070007BE00E94652DBC016C5D754077FF03C05D
:10208000719561957109882777FD8095982F0E9439
:102090009B2A2EE333EC4EE259E30E94AB2B20E067
:1020A00030E040EC5EE30E94982960930601709353
:1020B0000701809308019093090189C010922B02B7
:1020C00010922C0210922D0210922E02CE018370DB
:1020D0009927892BE1F0BE016170772780E090E0BD
:1020E0000E94992A20E030E040E05EE30E94AB2BA2
:1020F00020E030E040E45FE30E949829609306010D
:102100007093070180930801909309010CC080E04F
:1021100090E0A0E0BFE38093060190930701A093B5
:102120000801B0930901C770DD27CD2B09F04FC01E
:1021300010920601109207011092080110920901F5
:1021400046C010922B0210922C0210922D02109277
:102150002E0200E010E020E03FE300930601109320
:10216000070120930801309309016739710578F15F
:1021700080E090E00E94992A20E030E047E153E4BB
:102180000E94972920E030E04AE754E40E94002AA8
:1021900020E030E048E452E40E94AB2B20E030E045
:1021A00040EA51E40E94DD2A0E94682A660F771FE8
:1021B000660F771FFB01EE5AFE4F2081318142816D
:1021C0005381C701B6010E94AB2B6B017C01C70193
:1021D000B601DF91CF911F910F91FF90EF90DF90AB
:1021E000CF90BF90AF909F908F90089580918C0278
:1021F0000895CF93DF9300D01F92CDB7DEB79C0137
:1022000080911303843019F593E099833B832A83EB
:102210009093E9008FEF9091E800815095FD06C002
:1022200095ED9A95F1F700008111F5CF8091E800C6
:1022300085FF0DC040E050E063E070E0CE01019604
:102240000E945A138091E8008E778093E8000F90E7
:102250000F900F90DF91CF910895CF93DF9300D02F
:102260001F92CDB7DEB720911303243021F522E071
:1022700029839B838A8383E08093E9008FEF909189
:10228000E800815095FD06C095ED9A95F1F70000A4
:102290008111F5CF8091E80085FF0DC040E050E04E
:1022A00063E070E0CE0101960E945A138091E8002D
:1022B0008E778093E8000F900F900F90DF91CF9171
:1022C0000895209113032430F1F422E02093E900D3
:1022D0002FEF3091E800215035FD06C035ED3A95DD
:1022E000F1F700002111F5CF2091E80025FF0BC088
:1022F00040E050E065E070E00E945A138091E800F1
:102300008E778093E8000895CF93DF93EC0190914E
:102310001303943009F046C0809115018823D9F049
:10232000809116018823B9F09093E9008FEF909186
:10233000E800815095FD06C095E19A95F1F70000FF
:102340008111F5CF8091E80085FF2CC040E050E07E
:1023500060E170E017C081E08093E9008FEF909119
:10236000E800815095FD06C095ED9A95F1F70000C3
:102370008111F5CF8091E80085FF14C040E050E066
:1023800068E070E0CE010E945A138091E8008E77D9
:102390008093E80080E1FE01ACE7B2E001900D928D
:1023A0008A95E1F7DF91CF91089580911203811111
:1023B00009C00E94EF140E944C158091E2008460D5
:1023C0008093E200089510921203089508950895ED
:1023D0000C94932342E061EC81E00E94691442E096
:1023E00061EC82E00E94691442E061EC83E00E94AB
:1023F000691442E161EC84E00C9469148091150346
:10240000833009F455C030F4813071F0823009F422
:102410008EC008958A3009F47AC08B3009F460C008
:10242000893009F09CC020C080911403813A09F0E2
:1024300096C08091E800877F8093E8008091180320
:1024400090911903892B21F460E18CE792E003C09D
:1024500060E080E090E070E00E94A5138091E800C9
:102460008B778093E800089580911403813209F0FE
:1024700076C08091180390911903009719F0039783
:1024800009F06DC08091E800877F8093E80080911B
:10249000E80082FD05C0809113038111F8CF5FC071
:1024A0008091F10080938C028091E8008B7753C07B
:1024B00080911403813A09F052C0809118039091E1
:1024C0001903892B09F04BC08091E800877F809326
:1024D000E8008091E80080FFFCCF8091150136C0B4
:1024E000809114038132D9F58091180390911903DA
:1024F000892BA9F58091E800877F8093E8000E94EE
:102500009E1480911603809315010C94D41C809125
:102510001403813221F58091E800877F8093E800E1
:102520000E949E148091170380938D0208958091DC
:102530001403813AA1F48091E800877F8093E8003A
:102540008091E80080FFFCCF80918D028093F100A4
:102550008091E8008E778093E8000C949E14089593
:1025600084B7877F84BF88E10FB6F89480936000BA
:10257000109260000FBE90E080E80FB6F894809350
:102580006100909361000FBE0E9441180E94EF14F9
:102590000E944C158091E20084608093E200789460
:1025A0000E94D2170E9443188BE091E00E94ED1721
:1025B00080911303853069F40E94542380911103A4
:1025C0008823B1F30E948223882391F30E9444134D
:1025D000EFCF0E944B18ECCF292F33272330310542
:1025E000C9F064F42130310581F02230310509F061
:1025F00043C08DE690E024E535E042C0213231054C
:10260000F1F02232310541F137C082E190E021EC56
:1026100035E036C099278130910541F0823091052F
:1026200041F0892B49F5E0E5F5E005C0E2E2F5E08F
:1026300002C0E8EFF4E0849190E09F0121C0643093
:10264000D8F4E62FF0E0EE0FFF1FE255FE4F208199
:10265000318189E090E014C0643070F470E0FB01D7
:10266000EE0FFF1FEA55FE4F20813181FB01EE5531
:10267000FE4F808190E004C080E090E020E030E0F8
:10268000FA0131832083089580E189BD82E189BD0B
:1026900009B400FEFDCF8091D8008F7D8093D800D3
:1026A0008091E00082608093E0008091E00081FDF5
:1026B000FCCF0895CF92DF92EF92FF920F931F937A
:1026C000CF93DF93EC018B016A010E94BD1481114D
:1026D00033C0C114D10439F0F60180819181081B07
:1026E000190BC80FD91FE12CF12C0115110519F197
:1026F0008091E80085FD16C08091E8008E77809378
:10270000E800C114D10449F0F60180819181E80EFE
:10271000F91EF182E08285E00FC00E94BD1488237B
:1027200021F30AC089918093F10001501109FFEF54
:10273000EF1AFF0ADACF80E0DF91CF911F910F915E
:10274000FF90EF90DF90CF90089520911A03309181
:102750001B032617370748F06115710539F42091DE
:10276000E8002E772093E80001C0B90140E0611530
:102770007105A9F120911303222309F443C02530E8
:1027800009F442C02091E80023FD40C02091E800F8
:1027900022FD32C02091E80020FFE9CF4091F300F4
:1027A0002091F20030E0342BFC01CF01611571055E
:1027B00059F02830310540F481918093F100615047
:1027C00071092F5F3F4FF1CF41E02830310509F00B
:1027D00040E02091E8002E772093E800C8CF411117
:1027E000C9CF0AC080911303882361F0853061F05E
:1027F0008091E80083FD0AC08091E80082FFF2CF5B
:1028000080E0089582E0089583E0089581E00895CE
:1028100020911A0330911B032617370748F06115E2
:10282000710539F42091E8002E772093E80001C06B
:10283000B901FC0120E06115710591F1809113034C
:10284000882309F440C0853009F43FC08091E80036
:1028500083FD3DC08091E80082FD2FC08091E8009B
:1028600080FFE9CF2091F3008091F20090E0922B5D
:102870006115710559F08830910540F42491209339
:10288000F1003196615071090196F2CF21E008976D
:1028900009F020E08091E8008E778093E800CBCFAC
:1028A0002111CCCF0AC080911303882361F08530B9
:1028B00061F08091E80083FD0AC08091E80082FF0A
:1028C000F2CF80E0089582E0089583E0089581E0EA
:1028D0000895982F973058F59093E900981739F09C
:1028E0007091EC002091ED005091F00003C0242F76
:1028F000762F50E021FF19C03091EB003E7F3093DE
:10290000EB003091ED003D7F3093ED003091EB0016
:1029100031603093EB007093EC002093ED00509306
:10292000F0002091EE0027FF07C09F5FD3CF8F708C
:102930008093E90081E0089580E008958091140378
:1029400087FF11C08091E80082FD05C080911303CC
:102950008111F8CF11C08091E8008B770BC0809176
:102960001303882349F08091E80080FFF8CF80911D
:10297000E8008E778093E80008952091E40030917C
:10298000E50095E64091EC00842F817040FF22C065
:102990008091E80080FD1CC080911303882391F092
:1029A000853091F08091EB0085FD10C04091E400EE
:1029B0005091E5004217530729F39A01915011F7FE
:1029C00084E0089582E0089583E0089581E0089509
:1029D00080E008954091E80042FFDECF08950E9414
:1029E0005D150E946515E0EEF0E0808181608083D6
:1029F000E8EDF0E080818F77808319BCA7EDB0E02F
:102A00008C918E7F8C9380818F7E808310921203B5
:102A100008950F931F93CF93DF930E945D150E943B
:102A20006515C8EDD0E088818F77888388818068BC
:102A3000888388818F7D888319BC1092130310923C
:102A40000F03109211031092100300EE10E0F80132
:102A500080818B7F808388818160888342E060E011
:102A600080E00E946914E1EEF0E080818E7F808337
:102A7000E2EEF0E0808181608083808188608083E5
:102A8000F80180818E7F8083888180618883DF91D7
:102A9000CF911F910F910895E8EDF0E080818F7E36
:102AA0008083E7EDF0E080818160808384E082BFF5
:102AB00081E0809312030C940915E8EDF0E0808129
:102AC0008E7F80831092E20008951092DA001092B7
:102AD000E10008951F920F920FB60F9211242F93C9
:102AE0003F934F935F936F937F938F939F93AF9396
:102AF000BF93EF93FF938091E10082FF0BC0809121
:102B0000E20082FF07C08091E1008B7F8093E100AB
:102B10000E94D1178091DA0080FF1FC08091D800F9
:102B200080FF1BC08091DA008E7F8093DA00809155
:102B3000D90080FF0DC080E189BD82E189BD09B463
:102B400000FEFDCF81E0809313030E94D51105C0E4
:102B500019BC109213030E94E3118091E10080FFE1
:102B600019C08091E20080FF15C08091E2008E7F45
:102B70008093E2008091E20080618093E200809186
:102B8000D80080628093D80019BC85E0809313033D
:102B90000E94E7118091E10084FF30C08091E20043
:102BA00084FF2CC080E189BD82E189BD09B400FEAB
:102BB000FDCF8091D8008F7D8093D8008091E10077
:102BC0008F7E8093E1008091E2008F7E8093E2000F
:102BD0008091E20081608093E20080910F0388235E
:102BE00011F084E007C08091E30087FD02C081E01E
:102BF00001C083E0809313030E94E8118091E100FB
:102C000083FF29C08091E20083FF25C08091E1000D
:102C1000877F8093E10082E08093130310920F037B
:102C20008091E1008E7F8093E1008091E2008E7FB1
:102C30008093E2008091E20080618093E20042E0B4
:102C400060E080E00E9469148091F00088608093C9
:102C5000F0000E94E611FF91EF91BF91AF919F911B
:102C60008F917F916F915F914F913F912F910F9035
:102C70000FBE0F901F9018951F920F920FB60F92D4
:102C800011242F933F934F935F936F937F938F9371
:102C90009F93AF93BF93CF93DF93EF93FF93C09135
:102CA000E900CF708091EC00D82FD17080FDD0E882
:102CB0001092E9008091F000877F8093F000789473
:102CC0000E9480161092E9008091F0008860809345
:102CD000F000CD2BCF70C093E900FF91EF91DF9111
:102CE000CF91BF91AF919F918F917F916F915F91A4
:102CF0004F913F912F910F900FBE0F901F901895FD
:102D00001F93CF93DF93CDB7DEB7AA970FB6F89492
:102D1000DEBF0FBECDBFE4E1F3E088E08E0F9091FF
:102D2000F10091938E13FBCF0E94FE118091E80079
:102D300083FF1FC18091140390911503492F50E028
:102D40004A30510508F015C1FA01EA5AFF4F0C94B8
:102D50008D2D803881F0823809F00BC180911803E5
:102D60008F708093E9008091EB0085FB882780F9C4
:102D70001092E90006C08091100390911103911107
:102D800082609091E800977F9093E8008093F10033
:102D90001092F100C8C0282F2D7F09F0EAC08823C7
:102DA00019F0823061F0E5C080911603813009F09E
:102DB000E0C0933009F080E0809311032BC0809134
:102DC0001603811127C0809118038F7009F4D1C0B8
:102DD0008093E9002091EB0020FF1CC0933021F488
:102DE0008091EB00806214C09091EB009061909311
:102DF000EB0021E030E0A90102C0440F551F8A9585
:102E0000E2F74093EA001092EA008091EB008860BC
:102E10008093EB001092E9008091E800877F86C0E4
:102E20008111A7C0109116031F778091E30080786D
:102E3000812B8093E3008091E800877F8093E800F6
:102E40000E949E148091E80080FFFCCF8091E300F7
:102E500080688093E300111102C082E001C083E02A
:102E60008093130386C08058823008F082C080911E
:102E70001603909117038C3D53E0950779F583E095
:102E80008A838AE289834FB7F894DE01139620E0A3
:102E90003EE051E2E32FF0E050935700E49120FF31
:102EA00003C0E295EF703F5FEF708E2F90E0EA3045
:102EB00010F0C79601C0C0968D939D932F5F24316B
:102EC00049F74FBF8091E800877F8093E8006AE26E
:102ED00070E0CE0101960E94A51314C0AE014F5FB1
:102EE0005F4F609118030E94EC12BC01009709F437
:102EF00040C09091E800977F9093E80089819A8183
:102F00000E9408148091E8008B778093E80031C01C
:102F1000803879F58091E800877F8093E800809180
:102F20000F038093F1008091E8008E778093E80092
:102F30000E949E141EC081111CC0909116039230F5
:102F4000C0F48091E800877F8093E80090930F039E
:102F50000E949E1480910F03811106C08091E300AE
:102F600087FD02C081E001C084E0809313030E94CA
:102F7000EA118091E80083FF0AC08091E800877F12
:102F80008093E8008091EB0080628093EB00AA962A
:102F90000FB6F894DEBF0FBECDBFDF91CF911F916A
:102FA00008950895CF93809113038823A1F0C091D1
:102FB000E900CF709091EC00892F817090FD80E83E
:102FC000C82B1092E9008091E80083FD0E948016D2
:102FD000CF70C093E900CF910895909393028093AE
:102FE00092020895E0919202F0919302309721F0BD
:102FF0000190F081E02D099480E00895E091920223
:10300000F0919302309721F00280F381E02D099432
:103010000895E0919202F0919302309721F004809C
:10302000F581E02D0994089520919002309191024C
:103030008217930771F09093910280939002E09130
:103040009202F0919302309721F00680F781E02DF3
:103050000994089520918E0230918F028217930770
:1030600071F090938F0280938E02E0919202F09122
:103070009302309721F00084F185E02D09940895A2
:1030800008950C9440180E94C7230E94180A0E94B9
:103090004D240C94FC285F926F927F928F929F92A6
:1030A000AF92BF92CF92DF92EF92FF920F931F9356
:1030B000CF93DF9300D000D01F92CDB7DEB70E9430
:1030C0005D0A9DE9C92E92E0D92E03E010E0AA2402
:1030D000A394B12C502E802F0E94D80A4C01F601E7
:1030E000729062906F016826792661147104A1F4D0
:1030F0000150110978F78FEF89838A831B820E9420
:10310000D0238160782F9D838C8349815A816B8184
:103110008D810E94FB1838C08091F20281FD0E94CF
:10312000E10A2BE030E07501022E02C0EE0CFF1C1C
:103130000A94E2F7C70186219721892B09F1298397
:103140005A828E209F2091E0892809F490E09B8389
:103150000E94D0238160782F9D838C8349815A817E
:103160006B818D810E94FB18000F111FF801EB5637
:10317000FD4F80819181E826F926F182E08204C02A
:103180002150310980F6B4CF0E9434261091940268
:103190000E94F2171817D1F00E94F2178093940240
:1031A0000F900F900F900F900F90DF91CF911F9184
:1031B0000F91FF90EF90DF90CF90BF90AF909F90D6
:1031C0008F907F906F905F900C94020A0F900F90F9
:1031D0000F900F900F90DF91CF911F910F91FF9063
:1031E000EF90DF90CF90BF90AF909F908F907F90A7
:1031F0006F905F900895CF93DF93CDB7DEB72B9795
:103200000FB6F894DEBF0FBECDBF4F8358876987D6
:103210007A878B87DE01119686E0FD0111928A95EF
:10322000E9F785E0FE01379601900D928A95E1F766
:1032300049815A816B817C818D819E810E94721FA0
:103240002B960FB6F894DEBF0FBECDBFDF91CF91A6
:103250000895CF93882309F4C2C0C82F823859F447
:103260000E94F21781FDBBC089E30E944C220E949C
:10327000192389E30CC0833879F40E94F21780FD8A
:10328000AEC083E50E944C220E94192383E50E9470
:103290008E22CF910C941923843859F40E94F2178E
:1032A00082FD9DC087E40E944C220E94192387E47E
:1032B000EECF8CEF8C0F813A48F48C2F0E9464285B
:1032C00081118DC08C2F0E944C22E3CF80E28C0FA5
:1032D000883048F4C77081E001C0880FCA95EAF7CA
:1032E0000E94D222D6CF8BE58C0F833078F4C53A7A
:1032F00029F0C63A31F083E890E005C081E890E01B
:1033000002C082E890E0CF910C94141888E58C0FED
:10331000833108F064C0C83A39F1C93A41F1CA3A78
:1033200049F1CB3A51F1CC3A59F1CD3A61F1C03B78
:1033300069F1CE3A71F1CF3A79F1C13B81F1C23BEB
:1033400089F1C33B91F1C43B99F1C53BA1F1C63B67
:10335000A9F1C73BB1F1C83BB9F1C93BC1F1CA3BC7
:10336000C9F180E090E038C082EE90E035C089EE8F
:1033700090E032C08AEE90E02FC085EB90E02CC048
:1033800086EB90E029C087EB90E026C08CEC90E0C3
:1033900023C08DEC90E020C083E891E01DC08AE856
:1033A00091E01AC082E991E017C084E991E014C06D
:1033B00081E292E011C083E292E00EC084E292E0EA
:1033C0000BC085E292E008C086E292E005C087E289
:1033D00092E002C08AE292E0CF910C942A18CF9139
:1033E0000895882309F44BC0823859F40E94F217DB
:1033F00081FF45C089E30E944C220E94192389E382
:103400000CC0833871F40E94F21780FF38C083E546
:103410000E944C220E94192383E50E948E220C9464
:103420001923843859F40E94F21782FF28C087E4D8
:103430000E944C220E94192387E4EFCF9CEF980F43
:10344000913A58F390E2980F983050F4877091E0D9
:1034500001C0990F8A95EAF7892F0E94D822DFCF01
:103460009BE5980F933020F480E090E00C941418C2
:10347000885A833120F480E090E00C942A18089553
:10348000882321F00E94D2220C94192308958823C6
:1034900021F00E94D8220C94192308957F928F92D4
:1034A0009F92AF92BF92CF92DF92EF92FF920F93D3
:1034B0001F93CF93DF931F92CDB7DEB77C01C62E4B
:1034C000772EFC01058102950F70128111110E9467
:1034D000EF220E944522882379F0112369F080E2CF
:1034E0008C0D883048F082E00E942E220E944522F6
:1034F00091E0D82ED92601C0D12CE72DE295EF70AE
:10350000F0E0E05AFF4F0C948D2D872D807F072D22
:103510000F70882311F00295007F112389F000239A
:1035200009F499C180E28C0D883020F4802F0E942C
:10353000D22203C0802F0E94E2220E9419238BC155
:103540008C2D0E94F119002309F4C3C180E28C0D77
:10355000883020F4802F0E94D82203C0802F0E9440
:10356000E8220E941923B5C1872D807F972D9F7077
:10357000803211F4892F03C0892F8295807FCC205F
:1035800021F0F1E0CF16A1F01DC0112339F0002386
:1035900019F1013009F50E9402239BC1002319F0A3
:1035A000013009F496C189830E940523898110C1E5
:1035B000112321F0063008F08CC10EC0053008F050
:1035C00088C106C1112359F0002331F0F70195811C
:1035D00090FF41C19F7095830E94401A7AC10023D9
:1035E00009F4F6C03EC1872D86958695837090E0DC
:1035F000009719F0019761F06CC1112321F08C2D17
:10360000972D937002C080E090E00E94141861C171
:10361000112321F08C2D972D937002C080E090E053
:103620000E942A1856C18C2D112319F00E943C25A6
:1036300002C00E94A4250E9429264BC1872D8370B9
:1036400009F052C0111145C18C2D82958695877065
:10365000880F880F9C2D9F70892E912CA12CB12C46
:10366000082E04C0880C991CAA1CBB1C0A94D2F713
:10367000C4FE14C00FE010E020E030E0B901A80162
:1036800004C0440F551F661F771F8A95D2F7CB01E0
:10369000BA01609570958095909503C060E070E0E8
:1036A000CB01272D26952695237030E02230310559
:1036B00069F02330310589F0682979298A299B2905
:1036C0002130310571F00E94BA2003C1682979299F
:1036D0008A299B290E94D620FCC00E94BA20C501DD
:1036E000B4010E949E20F5C0112319F0872D81702E
:1036F00001C08695882309F4ECC08C2D82958695AF
:103700008770880F880F9C2D9F70892E912CA12C7B
:10371000B12C082E04C0880C991CAA1CBB1C0A944E
:10372000D2F7C4FE14C00FE010E020E030E0B90191
:10373000A80104C0440F551F661F771F8A95D2F752
:10374000CB01BA01609570958095909503C060E0BB
:1037500070E0CB01272D269526952370422F50E04F
:103760004230510569F04330510589F068297929C3
:103770008A299B294130510571F00E949421A9C0EA
:10378000682979298A299B290E94B021A2C00E9418
:103790009421C501B4010E9478219BC08C2D90E03A
:1037A000FC01E05EF109E531F10508F050C0E05997
:1037B000FF4F0C948D2D0C2D0F70872D8F711123C1
:1037C00021F00E941121802F07CF0E943221802FEB
:1037D0000E94471A7EC0112341F0053008F079C0DD
:1037E000872D8F710E94572174C0063008F071C078
:1037F000F7CF112339F0872D8F710E94112169C0F5
:103800001123C9F3872D8F710E94322162C01123C9
:1038100029F0872D8F710E94FC205BC00E94F2204E
:1038200058C0112351F0172D1F71812F0E941121B3
:1038300063E0812F0E9425224CC081E00E942E224D
:10384000023008F446C082E00E942E2242C01123BA
:1038500031F0002381F28C2D0E9429193AC00023F7
:1038600089F28C2D0E94F11934C0472D4F706C2DB8
:10387000C7010E945B040E9416202BC0111129C0B1
:10388000472D4F7050E042305105B9F04CF44115CE
:10389000510581F041305105E1F40E94242919C0FD
:1038A0004330510569F04430510599F48C2D0E9444
:1038B00076290FC00E940D290CC00E94402909C022
:1038C0000E94532906C0472D4F706C2DC7010E94DE
:1038D000E306DD20F9F00E94212280FD1BC0F701E4
:1038E00012820E941B220E941121C7010E94991C72
:1038F0000E941B220F90DF91CF911F910F91FF909B
:10390000EF90DF90CF90BF90AF909F908F907F907F
:103910000C9432210F90DF91CF911F910F91FF9066
:10392000EF90DF90CF90BF90AF909F908F907F905F
:1039300008950F931F93CF93DF93EC0188819981B2
:103940002B813C81232BB9F09F3F11F48F3F99F0DD
:10395000CE010E94E204882371F0688179818A8116
:103960000E9417228C010E94CC210E949320B80152
:10397000CE010E944E1ADF91CF911F910F910895B1
:103980000E94EF220E94FF220E94C4220E9419235B
:103990000E94DA260E94292680E090E00E941418F6
:1039A00080E090E00C942A180E94DF220C94C01C46
:1039B0000E940C22292F22952F7030E02C303105E7
:1039C0004CF42A3031056CF4225031092230310593
:1039D000A8F407C02C30310569F02F30310551F0C3
:1039E0000DC0803F69F018F4803E40F409C0843F68
:1039F00029F406C093FB882780F9089580E0089594
:103A000081E00895CF93DF9300D000D01F92CDB70F
:103A1000DEB70F900F900F900F900F90DF91CF9126
:103A20000895CF93DF9300D000D000D0CDB7DEB79C
:103A300026960FB6F894DEBF0FBECDBFDF91CF91B3
:103A400008951F93CF93DF93C0919D0216E080915C
:103A50009E02C81799F0D0E01C9FF0011D9FF00D49
:103A60001124E156FD4F408151816281738184812F
:103A700095810E94111D2196C770E9CFDF91CF91EA
:103A80001F9108954091CF025091D0026091D102D0
:103A90007091D2028091D3029091D4020C94111DA6
:103AA0008091D40282958F7009F054C08091D10228
:103AB000882309F44FC080919D02A0919E026091DD
:103AC000CF027091D0024091D2025091D302B6E061
:103AD0008A1709F43FC090E041155105C1F17F3FBD
:103AE00011F46F3FA1F1B89FF001B99FF00D1124BF
:103AF000E156FD4F218172132AC02081621327C035
:103B00002281211124C0238134812417350710F428
:103B100021503109241B350B283C3105C0F420917C
:103B2000D4022F7020612093D40226E0289FF00158
:103B3000299FF00D1124EC55FD4F80818F7080611D
:103B400080838FEC92E00E94991C0C94211D0196B9
:103B50008770BECF0895CF92DF92EF92FF920F93BE
:103B60001F93CF93DF93CDB7DEB762970FB6F8946C
:103B7000DEBF0FBECDBF8C0185E0F801DE011D96D2
:103B800001900D928A95E1F7D8014C9111965C91C4
:103B9000119712966C9112971396CD90DC90149712
:103BA0003091CF027091D0028091D2029091D302D5
:103BB000009709F46BC17F3F19F43F3F09F466C1D8
:103BC000E090D102EE2009F4C0C02091D402C816C2
:103BD000D90628F0F601E81BF90BCF0104C0809547
:103BE00090958C0D9D1DFF24F394883C910578F0F1
:103BF000F12C207F09F0C6C07C2DD98AC88A89891A
:103C00000E94021D8FEC92E00E94991CB1C0822F8D
:103C1000807F09F046C0751314C0341312C06111BF
:103C200010C02F7020612093D4020E94421D8FEC9F
:103C300092E00E94991C8091D402D80115968C9331
:103C40002EC0CD2819F15F3F11F44F3FF9F0F62E49
:103C500061111CC080919D0220919E0236E0821766
:103C600009F45AC090E0389FF001399FF00D1124FB
:103C7000E156FD4F7181571306C07081471303C091
:103C80007281711103C001968770E9CFF62E662309
:103C900009F418C18091D40281608093D402F12C80
:103CA00011C1751308C0341306C0611104C080919E
:103CB000D402D801C3C04D875E878D859E856A8BEF
:103CC0000E94D81C6A898823E1F16623D1F12091F2
:103CD000D402822F82958F7090E0029774F08091C9
:103CE000CF029091D00298878F831986DB86CA868F
:103CF0002C87CE0107960E94991C86E0F801AFEC54
:103D0000B2E001900D928A95E1F70E94501D0E9449
:103D1000421DFF24F394D6C04D875E878D859E8516
:103D20000E940C22292F22952F7030E0223031057D
:103D30000CF0BCC09F7009F0B6C0805E883008F4FB
:103D4000C1C0C8010E94991CE4CFC816D90608F466
:103D500053C0F601E81BF90BCF01883C910508F42C
:103D600050C0F12C7C2DD98AC88A89890E94021DF5
:103D7000EFECF2E086E0DF011D928A95E9F70E9400
:103D8000421DA0C0751314C0341312C0611110C0BD
:103D90008091D402F8018583C8010E94991C86E0B5
:103DA000EFECF2E0DF011D928A95E9F7FE2C8AC064
:103DB0004D875E878D859E856A8B0E94D81C6A8997
:103DC000882309F4BECF662309F4BBCF2091D40227
:103DD000822F82958F7090E002970CF48ECF8091A5
:103DE000CF029091D0029A8389831B82DD82CC829C
:103DF0002E83CE0101967FCF809590958C0D9D1DD1
:103E0000ACCFF62E662309F49CCF75132EC0341365
:103E10002CC02091D40220FD1FC0822F82958F706C
:103E2000D9F0D80115962C9315978F3049F08F5FF4
:103E3000982F9295907F822F8F70892B15968C9357
:103E4000C8010E94991C86E0F801AFECB2E0019035
:103E50000D928A95E1F793CF86E0F801AFECB2E0DE
:103E600001900D928A95E1F72DC04D875E878D8573
:103E70009E850E94D81C811140CF8091D402816020
:103E80008093D402C8010E94991C1CC0662309F4C7
:103E900058CF4D875E878D859E850E94D81C8823CC
:103EA00009F44FCF2ACF811148CF0CC024303105FF
:103EB0000CF047CF9F7009F440CFF8019581907FB7
:103EC00009F03BCF8F2D62960FB6F894DEBF0FBE80
:103ED000CDBFDF91CF911F910F91FF90EF90DF90B9
:103EE000CF9008951F93CF93DF93CDB7DEB72C9774
:103EF0000FB6F894DEBF0FBECDBF4F8358876987DA
:103F00007A878B879C87CE0107960E94AB1D8823FA
:103F100069F08F8198852A853B85232BF1F19F3F9E
:103F200009F063C08F3F09F060C037C086E0FE0132
:103F30003796DE01119601900D928A95E1F76F8117
:103F40007885EA85FB85309741F17F3F11F46F3F1B
:103F500021F120919E0230E0C901019687709927D6
:103F600040919D0250E08417950709F447C069838A
:103F70007A83FD83EC8396E0929FD001939FB00DEE
:103F80001124A156BD4FFE01319601900D929A95D4
:103F9000E1F780939E020E94211D16E080919D0210
:103FA00090919E028917C1F1189FC001112481567A
:103FB0009D4F0E94AB1D882379F1E0919D021E9FC9
:103FC000F0011124E156FD4F4081518162817381DE
:103FD000848195810E94111D80919D0290E001963F
:103FE0008770992780939D02D9CF4F815885698525
:103FF0007A858B859C850E94111DCFCF0E94D41C91
:1040000010929E0210929D02EFECF2E086E0DF013A
:104010001D928A95E9F7C1CF2C960FB6F894DEBFB2
:104020000FBECDBFDF91CF911F910895EF92FF9208
:104030000F931F93CF93DF938C01009709F46CC00B
:10404000F12CEE24E394E8012196F8018491843761
:1040500040F4843008F051C0813081F0823019F191
:104060005BC0853709F444C0A8F19CE7980F9037EE
:1040700008F052C08F770E94F11941C00E5F1F4FA8
:10408000FE01C49180E28C0F883048F4C7708E2DF9
:1040900001C0880FCA95EAF70E94F22214C08C2F43
:1040A0000E9429192DC00E5F1F4FFE01C49180E2AE
:1040B0008C0F883058F4C7708E2D01C0880FCA95B8
:1040C000EAF70E94F8220E9419231AC08C2F0E943E
:1040D000F11916C00E5F1F4FFE01C491CC2381F071
:1040E0008FE99FE00197F1F700C00000C150F6CFC3
:1040F0000E5F1F4FFE01F49003C00E9429198E012C
:104100008F2D882309F49FCFEFE9FFE03197F1F776
:1041100000C000008150F5CFDF91CF911F910F912A
:10412000FF90EF90089508956093D9027093DA029A
:104130008093DB029093DC020C94C01C0F931F93BE
:104140000091D9021091DA022091DB023091DC0259
:10415000DC01CB01802B912BA22BB32B8093D902B6
:104160009093DA02A093DB02B093DC021F910F91CF
:104170000C94C01C0F931F930091D9021091DA0286
:104180002091DB023091DC02DC01CB018023912302
:10419000A223B3238093D9029093DA02A093DB0287
:1041A000B093DC021F910F910C94C01C0F931F93CE
:1041B0000091D9021091DA022091DB023091DC02E9
:1041C000DC01CB0180279127A227B3278093D90256
:1041D0009093DA02A093DB02B093DC021F910F915F
:1041E0000C94C01C1092D5021092D6021092D702E5
:1041F0001092D8020C94C01C41E050E060E070E0E6
:1042000004C0440F551F661F771F8A95D2F740934D
:10421000D5025093D6026093D7027093D8020C94C3
:10422000C01C41E050E060E070E004C0440F551F46
:10423000661F771F8A95D2F78091D5029091D6029A
:10424000A091D702B091D802482B592B6A2B7B2B17
:104250004093D5025093D6026093D7027093D80250
:104260000C94C01C41E050E060E070E004C0440FDA
:10427000551F661F771F8A95D2F740955095609518
:1042800070958091D5029091D602A091D702B091FD
:10429000D802482359236A237B234093D5025093A5
:1042A000D6026093D7027093D8020C94C01C41E0F0
:1042B00050E060E070E004C0440F551F661F771F98
:1042C0008A95D2F78091D5029091D602A091D7021B
:1042D000B091D802482759276A277B274093D502F7
:1042E0005093D6026093D7027093D8020C94C01CEE
:1042F0000F931F930091D5021091D6022091D702FF
:104300003091D802DC01CB01802B912BA22BB32B57
:104310008093D5029093D602A093D702B093D8028F
:104320001F910F910C94C01C0F931F930091D50205
:104330001091D6022091D7023091D802DC01CB0136
:1043400080239123A223B3238093D5029093D60296
:10435000A093D702B093D8021F910F910C94C01C68
:104360000F931F930091D5021091D6022091D7028E
:104370003091D802DC01CB0180279127A227B327F7
:104380008093D5029093D602A093D702B093D8021F
:104390001F910F910C94C01C0895CF92DF92EF9261
:1043A000FF920F931F93CF93DF938C01C090D9029C
:1043B000D090DA02E090DB02F090DC028091D5022E
:1043C0009091D602A091D702B091D802C82AD92ADA
:1043D000EA2AFB2ACFE1D0E0D701C6010C2E04C0A7
:1043E000B695A795979587950A94D2F780FF06C052
:1043F000B8018C2F0E946809019721F4219760F77A
:1044000080E001C08C2FDF91CF911F910F91FF9021
:10441000EF90DF90CF900895CF93DF93EC010E944F
:10442000CD21BE010E946809DF91CF910895CB0193
:104430000E940C2208958091DD02859585958595D1
:1044400008958091DD028770089598E0899F90011A
:104450001124262B2093DD020C9411212091DD02E2
:10446000809582238093DD02982F977069F430E065
:10447000482F552747FD50952417350729F0859576
:10448000859585950C94322108959091DD02977061
:1044900081E009F480E0089590911501992321F0BD
:1044A00090911601911109C02091170130911801C6
:1044B000F90132969FEF40E01FC0982F9695969590
:1044C00096959F3050F5E0911701F0911801E90F92
:1044D000F11D877021E030E0A90102C0440F551F93
:1044E0008A95E2F7CA019181892B818308959F3FC4
:1044F00039F04F5F4E3041F051915813F8CF0DC055
:104500005111F7CF942FF5CF9F3F39F0F901E90F03
:10451000F11D97FDFA9582830895089590911501F4
:10452000992321F090911601911109C02091170152
:1045300030911801F9013296205F3F4F1FC0982F2C
:104540009695969596959F30F0F4E0911701F0912D
:104550001801E90FF11D877021E030E0A90102C0C8
:10456000440F551F8A95E2F7CA01809591818923EE
:10457000818308953196E217F30729F0908198130B
:10458000F9CF1082F7CF089581E090E0E091170114
:10459000F0911801E80FF91F108201968031910502
:1045A000A9F708959091F102892B8093F102089563
:1045B00080959091F10289238093F10208951092E1
:1045C000F10208959091F002892B8093F0020895F2
:1045D00080959091F00289238093F00208951092C3
:1045E000F00208959091EF02892B8093EF020895D5
:1045F00080959091EF0289238093EF0208951092A5
:10460000EF0208958093DE0208951092DE0208956D
:104610008091170190911801FC0131969C01205F57
:104620003F4F80E0919191118F5FE217F307D1F72F
:104630000895E0911701F09118018091F1028083B3
:10464000E0911701F091180190818091F002892B7F
:104650008083E0911701F091180190818091EF0221
:10466000892B80838091DE02882361F0E09117011D
:10467000F09118019081892B80830E940823811179
:104680001092DE0280911701909118010C94FE1790
:1046900020E0009739F0AC01415051098423952363
:1046A0002F5FF7CF822F089580911303843039F163
:1046B0001092F30220E488E190E00FB6F894A895F8
:1046C000809360000FBE2093600080E00E94C203D0
:1046D00080E00E94020A83B7817F846083BF83B732
:1046E000816083BF7894889583B78E7F83BF88E18C
:1046F0000FB6F89480936000109260000FBE08958A
:104700000895089580E00E94C2030E9480230E94C1
:104710005D0A0E9481230E94E20A91E0811101C09A
:1047200090E0892F08950E94D41C80E00E94C2036B
:104730000E94FC280E94F2170C94020A1F920F920A
:104740000FB60F9211248F939F93AF93BF938091D5
:10475000F302811113C08091F4029091F502A091AF
:10476000F602B091F7024196A11DB11D8093F402AB
:104770009093F502A093F602B093F702BF91AF9128
:104780009F918F910F900FBE0F901F90189582E010
:1047900084BD93E095BD9AEF97BD80936E00089518
:1047A0002FB7F8948091F4029091F502A091F6024F
:1047B000B091F7022FBF0895CF92DF92EF92FF9250
:1047C0000F931F932FB7F8944091F4025091F50284
:1047D0006091F6027091F7022FBF6A017B01EE240F
:1047E000FF248C0120E030E0C016D106E206F3067B
:1047F00010F4415051099A01281B390BC9011F912E
:104800000F91FF90EF90DF90CF9008951F920F923D
:104810000FB60F9211248F939F93AF93BF93809104
:10482000F4029091F502A091F602B091F702019680
:10483000A11DB11D8093F4029093F502A093F6029E
:10484000B093F702BF91AF919F918F910F900FBEE0
:104850000F901F9018950E94EF14F8942FEF87EA9D
:1048600091E6215080409040E1F700C0000087E0D1
:1048700090EBDC0180931E0390931F03A093200311
:10488000B09321039CE088E10FB6F894A89580933B
:1048900060000FBE90936000FFCF0E948C248111B6
:1048A00002C00E9468240E9497248093F2020E9412
:1048B0009F2480931C0387FB882780F9809316012F
:1048C0000E949B24682F70E080E090E00C9494207C
:1048D0006DEE7EEF80E090E00E94B32D60E082E01C
:1048E00090E00E94A12D60E083E090E00E94A12D65
:1048F00060E084E090E00E94A12D60E085E090E01F
:104900000E94A12D60E086E090E00E94A12D6FEF53
:1049100087E090E00C94A12D80E090E00E949B2D18
:1049200021E08D3E9E4F09F020E0822F089582E025
:1049300090E00C94932D83E090E00C94932D84E010
:1049400090E00C94932D682F84E090E00C94A12DBE
:1049500086E090E00C94932D682F86E090E00C9414
:10496000A12D87E090E00C94932D682F87E090E0D4
:104970000C94A12D8091FA0280FF0BC060911C0164
:1049800085E0689FB00111247595679575956795C9
:104990002BC081FF09C060911C0185E0689FB001B8
:1049A00011247595679520C082FF07C060911C0196
:1049B00085E0689FB001112417C09091FB029923F4
:1049C000D1F060911B01961788F720911C0185E0BA
:1049D000289F90011124929FA001939F500D1124B4
:1049E00070E0CA010E94792D6038710540F46115AC
:1049F000710539F002C065E070E0862F08958FE7F9
:104A0000089581E008958091FA0280FF08C06091C6
:104A10001A0170E0759567957595679521C081FFBE
:104A200006C060911A0170E07595679519C082FF04
:104A300004C060911A0170E010C09091FB029923AC
:104A4000C1F0609119019617A0F780911A01899F12
:104A5000C001112470E00E94792D6038710528F49E
:104A60006115710521F0862F08958FE7089581E083
:104A7000089561E070E0F4CF803F21F40E94BA24F1
:104A8000819504C0813F29F40E94BA248093FE02DC
:104A90000895823F21F40E94BA24819504C0833F87
:104AA00029F40E94BA248093FD020895893F19F4E5
:104AB0000E94032505C08A3F31F40E940325819599
:104AC0008093FF0208958B3F21F40E940325819576
:104AD00004C08C3F29F40E940325809300030895AD
:104AE000843F21F48091FC02816017C0853F21F44E
:104AF0008091FC02826011C0863F21F48091FC020B
:104B000084600BC0873F21F48091FC02886005C05F
:104B1000883F31F48091FC0280618093FC0208950B
:104B20008D3F21F48091FA0281600BC08E3F21F409
:104B30008091FA02826005C08F3F29F48091FA02C9
:104B400084608093FA020895803F39F48091FE02D8
:104B500087FF6CC01092FE0269C0813F29F48091EA
:104B6000FE021816BCF362C09091FD02823F29F448
:104B700097FF5CC01092FD0259C0833F19F41916CB
:104B8000CCF354C0893F41F48091FF0218160CF019
:104B90004DC01092FF024AC08A3F29F48091FF0263
:104BA00087FF44C0F6CF8B3F39F48091000387FF25
:104BB0003DC0109200033AC08C3F29F4809100035D
:104BC0001816BCF333C0843F21F48091FC028E7F21
:104BD00017C0853F21F48091FC028D7F11C0863F74
:104BE00021F48091FC028B7F0BC0873F21F48091E0
:104BF000FC02877F05C0883F31F48091FC028F7EE4
:104C00008093FC0213C08D3F21F48091FA028E7FC5
:104C10000BC08E3F21F48091FA028D7F05C08F3F3B
:104C200029F48091FA028B7F8093FA028091FD0231
:104C300081110EC08091FE0281110AC08091FF0295
:104C4000811106C080910003811102C01092FB0205
:104C500008958CEF92E00E9409180E94D02390934F
:104C6000F9028093F80208951F93CF93DF93809108
:104C7000F8029091F9020E94DC23AC019091FB02B2
:104C8000992321F020911D0130E006C020911E01E2
:104C90008AE0289F900111244217530708F486C028
:104CA0008091FD02C091FE02D091FF02109100039D
:104CB000811107C0C11176C0D11174C0111172C029
:104CC00075C09F3F19F09F5F9093FB02181624F464
:104CD0000E94BA248093FD028091FD0287FF05C0E7
:104CE0000E94BA2481958093FD021C1624F40E9430
:104CF000BA248093FE028091FE0287FF05C00E94C5
:104D0000BA2481958093FE026091FD02662339F1F9
:104D1000C091FE02CC2319F1772767FD7095872F8C
:104D2000972F0E949B2A23E333E343E35FE30E9430
:104D3000AB2B0E94682A6093FD026C2F772767FDDA
:104D40007095872F972F0E949B2A23E333E343E339
:104D50005FE30E94AB2B0E94682A6093FE021D163F
:104D600024F40E9403258093FF028091FF0287FFB5
:104D700005C00E94032581958093FF02111624F43B
:104D80000E940325809300038091000387FF05C0E4
:104D90000E940325819580930003DF91CF911F919D
:104DA0000C9429269F3F09F08ECF96CFDF91CF91AB
:104DB0001F910895ECEFF2E085E0DF011D928A95E6
:104DC000E9F71092FB021092FA020895833081F104
:104DD00028F4813059F08230D1F00895853009F4FB
:104DE00049C0B8F1863009F456C0089580911E017B
:104DF000262F30E0280F311D2F3F310524F4680F96
:104E000060931E0108958FEF80931E010895809195
:104E10001D01262F30E0280F311D2F3F310524F4CE
:104E2000680F60931D0108958FEF80931D01089511
:104E300080911C01262F30E0280F311D2F3F3105B6
:104E400024F4680F60931C0108958FEF80931C0178
:104E5000089580911B01262F30E0280F311D2F3F30
:104E6000310524F4680F60931B0108958FEF809340
:104E70001B01089580911A01262F30E0280F311D63
:104E80002F3F310524F4680F60931A0108958FEFC6
:104E900080931A01089580911901262F30E0280F80
:104EA000311D2F3F310524F4680F609319010895D7
:104EB0008FEF809319010895833011F128F4813028
:104EC00049F0823091F00895853081F120F18630EB
:104ED000C1F1089580911E01681720F4861B80930C
:104EE0001E01089510921E01089580911D016817FA
:104EF00020F4861B80931D01089510921D010895D2
:104F000080911C01681720F4861B80931C01089572
:104F100010921C01089580911B01681720F4861BD4
:104F200080931B01089510921B01089580911A012E
:104F3000681720F4861B80931A01089510921A01B5
:104F4000089580911901681720F4861B8093190138
:104F500008951092190108950F931F93873208F056
:104F600048C08E3108F08DC0803109F477C008F553
:104F7000873009F461C068F4863009F09DC08091E3
:104F8000F202817F8E7F8093F20281E080930203A0
:104F900094C08B3009F489C08E3009F08DC08091A7
:104FA000F20282FB222720F991E0922790FB82F9FE
:104FB0005EC0863109F479C060F4813109F07CC0AB
:104FC0000E94D41C9091160181E0892780931601DC
:104FD0006CC0893109F469C08B3109F06DC08091D2
:104FE000F20281FB222720F991E0922790FB81F9C0
:104FF0003EC0883309F459C050F4893209F457C0CF
:10500000853309F454C0873209F451C055C0833444
:1050100009F44DC028F48A3308F44EC0895332C0D5
:10502000883409F049C00E94D41C0E94120B0E94CF
:10503000D9040E942B2439C09091F202892F8095C7
:10504000817080FB90F929F0966098609093F2024D
:1050500034C0997F977F9093F20227C08091F2022B
:1050600083FB222720F991E0922790FB83F980931C
:10507000F2029923D1F08091F20281608093F202D2
:1050800014C08D5141E050E060E070E08A019B0166
:1050900004C0000F111F221F331F8A95D2F7C901C8
:1050A000B8010E9494200E94D41C81E006C061E0F7
:1050B00070E080E090E0F5CF80E01F910F910895BF
:1050C00080E0089580E00895CF93C82F8091020377
:1050D000813069F018F08230C9F184C0E091170185
:1050E000F09118018081823209F07EC007C0E09102
:1050F0001701F09118018081823261F48C2F0E9497
:105100006028811104C08C2F0E94AC271DC081E053
:1051100090E01AC08C2F0E946228811114C0C43103
:1051200079F048F4CB3079F0C03109F061C082E009
:105130008093020308C0C93219F0C83321F058C067
:105140001092020355C081E0817054C0C93291F1C0
:1051500020F5C43179F1B0F4C73009F047C08EE1D1
:1051600080931E0182E380931D018AE080931C01DD
:1051700084E180931B0188E080931A0188E2809388
:10518000190134C0CE51C63088F5EC2FF0E0EA5456
:10519000FE4F80818093010329C0CE34E9F020F4D2
:1051A000CB3421F56AE013C0C13579F0C235F1F492
:1051B00061E00DC080910103882319F01092010372
:1051C00015C081E08093020315C061E006C08091A4
:1051D00001030E94E6260AC06AE0809101030E9452
:1051E0005C2704C01092020380E004C081E002C08A
:1051F00080E0AACFCF9108950E948C24811102C033
:105200000E9468240E94A82480931D0380FF02C08E
:10521000869501C080E00C94C20380911D03982FF5
:105220009695292F30E0233031054CF49F5F990F7C
:105230008170892B816080931D030E94AC24809132
:105240001D0386950C94C20380911D03982F96959B
:1052500091F09158990F8170892B80931D038E7F57
:1052600091E009F490E080911D0390FB80F9809318
:105270001D030E94AC2480911D0386950C94C203EB
:1052800080911D03982F909590FB80F980931D03CA
:105290000E94AC2480911D0380FF02C0869501C04E
:1052A00080E00C94C20390911D03892F86958F5F37
:1052B0008F779170843028F4880F892B80931D0399
:1052C00002C090931D0380911D038E7F91E009F42D
:1052D00090E080911D0390FB80F980931D030E9454
:1052E000AC2480911D0386950C94C20320911D036C
:1052F000922F96958927982F990F822F8170892B4D
:1053000080931D038E7F91E009F490E080911D034E
:1053100090FB80F980931D030E94AC2480911D03B3
:1053200086950C94C20380911D038695089550586C
:10533000BB27AA270ED0D1C1C2D130F0C7D120F0EF
:1053400031F49F3F11F41EF4B7C10EF4E095E7FB72
:105350009FC1E92FD3D180F3BA176207730784077F
:10536000950718F071F49EF5EBC10EF4E0950B2E45
:10537000BA2FA02D0B01B90190010C01CA01A001A7
:105380001124FF27591B99F0593F50F4503E68F102
:105390001A16F040A22F232F342F4427585FF3CF43
:1053A000469537952795A795F0405395C9F77EF414
:1053B0001F16BA0B620B730B840BBAF09150A1F05D
:1053C000FF0FBB1F661F771F881FC2F70EC0BA0FE3
:1053D000621F731F841F48F4879577956795B7956B
:1053E000F7959E3F08F0B3CF9395880F08F0992763
:1053F000EE0F97958795089527D108F481E00895D9
:105400000CD06BC163D140F05AD130F021F45F3F32
:1054100019F03EC1511195C14FC170D198F3992334
:10542000C9F35523B1F3951B550BBB27AA27621768
:105430007307840738F09F5F5F4F220F331F441FAD
:10544000AA1FA9F333D00E2E3AF0E0E830D09150E5
:105450005040E695001CCAF729D0FE2F27D0660FD2
:10546000771F881FBB1F261737074807AB07B0E811
:1054700009F0BB0B802DBF01FF2793585F4F2AF027
:105480009E3F510568F004C15CC15F3FECF3983E5C
:10549000DCF3869577956795B795F7959F5FC9F784
:1054A000880F911D9695879597F90895E1E0660F0D
:1054B000771F881FBB1F621773078407BA0720F086
:1054C000621B730B840BBA0BEE1F88F7E0950895EF
:1054D00004D06894B11135C1089518D188F09F5750
:1054E00090F0B92F9927B751A0F0D1F0660F771F30
:1054F000881F991F1AF0BA95C9F712C0B13081F010
:105500001FD1B1E008951CC1672F782F8827B85F9D
:1055100039F0B93FCCF3869577956795B395D9F770
:105520003EF490958095709561957F4F8F4F9F4F7A
:105530000895E89409C097FB3EF490958095709586
:1055400061957F4F8F4F9F4F9923A9F0F92F96E9CF
:10555000BB279395F695879577956795B795F11144
:10556000F8CFFAF4BB0F11F460FF1BC06F5F7F4FE1
:105570008F4F9F4F16C0882311F096E911C07723F3
:1055800021F09EE8872F762F05C0662371F096E8FC
:10559000862F70E060E02AF09A95660F771F881FCB
:1055A000DAF7880F9695879597F9089588D018F0BF
:1055B00011F08CD038F480C0C4C0E92F9FD0B0F374
:1055C0005523C9F3E7FB6217730784079507A8F112
:1055D00099F3E92FFF2788232AF03197660F771F69
:1055E000881FDAF7952F5527442332F09150504009
:1055F000220F331F441FD2F7BB27E91BF50B621B99
:10560000730B840BB109C1F222F4620F731F841F64
:10561000B11D31972AF0660F771F881FBB1FEFCF90
:10562000915050405AF041F0882332F0660F771FB6
:10563000881F91505040C1F7939530C0869577955B
:1056400067959F5FD9F7F8CF990F0008550FAA0B00
:10565000E0E8FEEF16161706E807F907C0F0121685
:105660001306E407F50798F0621B730B840B950B88
:1056700039F40A2661F0232B242B252B21F40895DD
:105680000A2609F4A140A6958FEF811D811D08957A
:1056900097F99F6780E870E060E008959F3F31F0E0
:1056A000915020F4879577956795B795880F911D50
:1056B0009695879597F908959FEF80EC08950024BB
:1056C0000A941616170618060906089500240A9467
:1056D00012161306140605060895092E0394000CED
:1056E00011F4882352F0BB0F40F4BF2B11F460FF7C
:1056F00004C06F5F7F4F8F4F9F4F089557FD9058A5
:10570000440F551F59F05F3F71F04795880F97FB85
:10571000991F61F09F3F79F087950895121613063F
:105720001406551FF2CF4695F1DF08C0161617066E
:105730001806991FF1CF86957105610508940895A3
:10574000E894BB2766277727CB0197F908957CDF7C
:1057500008F48FEF08950BD0C0CFB1DF28F0B6DF8B
:1057600018F0952309F094CFA7CF1124EACFC6DF14
:10577000A0F3959FD1F3950F50E0551F629FF00164
:10578000729FBB27F00DB11D639FAA27F00DB11DBD
:10579000AA1F649F6627B00DA11D661F829F222746
:1057A000B00DA11D621F739FB00DA11D621F839FCD
:1057B000A00D611D221F749F3327A00D611D231FA3
:1057C000849F600D211D822F762F6A2F11249F57F1
:1057D00050408AF0E1F088234AF0EE0FFF1FBB1F14
:1057E000661F771F881F91505040A9F79E3F5105B3
:1057F00070F04ECFA6CF5F3FECF3983EDCF386957A
:1058000077956795B795F795E7959F5FC1F7FE2B5D
:10581000880F911D9695879597F90895FA01EE0FD7
:10582000FF1F30962105310599F16115710561F46D
:105830008038BFE39B0749F168949038810561F097
:105840008038BFEF9B0741F0992342F5FF3FE10508
:105850003105210511F1E8940894E795D901AA23AF
:1058600029F4AB2FBE2FF85FD0F310C0FF5F70F4A8
:10587000A695E0F7F73950F019F0FF3A38F49F7722
:105880009F930CD00F9007FC905808953EF014CFD2
:1058900060E070E080E89FE308954FE79F775F93B3
:1058A0004F933F932F939ED02F913F914F915F91B4
:1058B00052DF05C019F40EF0EBCE42CFFDCE26DF4D
:1058C000C8F39638C0F707F80F92E8942BE33AEA4A
:1058D00048EB5FE74EDF0F920F920F924DB75EB726
:1058E0000F92C0D0EAE0F1E016D04F915F91EF91B6
:1058F000FF91E595EE1FFF1F49F0FE57E068442732
:10590000EE0F441FFA95E1F74195550B32D00F90F9
:1059100007FE26C00895DF93CF931F930F93FF9246
:10592000EF92DF927B018C01689405C0DA2EEF01C3
:105930001EDFFE01E894A591259135914591559181
:10594000AEF3EF0106DDFE019701A801DA9479F7C5
:10595000DF90EF90FF900F911F91CF91DF9108950D
:105960009B01AC0160E070E080E89FE349CD90CE00
:1059700095CECCDEE8F39923D9F3940F511DBBF3F8
:105980009150504094F059F0882332F0660F771F01
:10599000881F91505040C1F79E3F510544F7880F32
:1059A000911D9695879597F908955F3FACF0983EC5
:1059B0009CF0BB27869577956795B79508F4B160FD
:1059C0009395C1F7BB0F58F711F460FFE8CF6F5FF5
:1059D0007F4F8F4F9F4FE3CFB4CE0EF05FCE6CCE94
:1059E000689456CE93DEC8F39923D1F3C6F3DF93C0
:1059F000CF931F930F93FF92C92FDD2788232AF09F
:105A00002197660F771F881FDAF720E030E040E823
:105A10005FEB9FE3883920F0803E30F021968F774E
:105A200087DCE2E3F1E003C083DCEFE5F1E073DF64
:105A30008B01BE01EC01FB2E6F5771097595771F25
:105A4000880B990B78DD28E132E741E35FE38FDED5
:105A5000AF2D9801AE01FF900F911F91CF91DF9173
:105A600078DC3BCEFA01DC01AA0FBB1F9B01AC0125
:105A7000BF5728F422273327442750781FC0B75137
:105A800088F4AB2F0024469537952795011CA395E4
:105A9000D2F3002069F0220F331F441FB395DAF3CD
:105AA0000DD045CC61307105A0E88A07B94630F4C5
:105AB0009B01AC016627772788279078309621F0E4
:105AC00020833183428353830895AA1BBB1B51E17A
:105AD00007C0AA1FBB1FA617B70710F0A61BB70B5E
:105AE000881F991F5A95A9F780959095BC01CD0103
:105AF000089597FB072E16F4009407D077FD09D080
:105B00000E94652D07FC05D03EF4909581959F4F2E
:105B10000895709561957F4F0895EE0FFF1F0590D2
:105B2000F491E02D0994F999FECF92BD81BDF89AC8
:105B3000992780B50895A8E1B0E042E050E00C94C8
:105B4000BB2D262FF999FECF92BD81BDF89A019702
:105B500000B4021639F01FBA20BD0FB6F894FA9AB5
:105B6000F99A0FBE08950196272F0E94A22D0C943A
:105B7000A12DDC01CB01FC01F999FECF06C0F2BDDD
:105B8000E1BDF89A319600B40D9241505040B8F7FB
:065B90000895F894FFCF18
:105B9600640007000CFF0000003F64F610841161EA
:105BA600112D11F9100101DF022808140A321E0016
:105BB60002040507090B0C0E1011131517181A1CF1
:105BC6001D1F2123242628292B2D2F30323435372B
:105BD600393B1F0F03764F5F6F7F49694379095938
:105BE60053633149803F5D8B803FF8BF803FCAE1F8
:105BF600803F73ED803FCAE1803FF8BF803F5D8BF9
:105C0600803F3149803F0000803FF16D7F3F75EA5C
:105C16007E3F4C827E3F833F7E3F84287E3F833F8C
:105C26007E3F4C827E3F75EA7E3FF16D7F3F0000EE
:105C3600803F3F4D36398F0642060C06D305660572
:105C46007F059805B105010203040506070809004A
:00000001FF
